:100000000C94AA010C94D2010C94D2010C94D2014C
:100010000C94D2010C94D2010C94D2010C94D20114
:100020000C94D2010C94D2010C9469070C94D8075B
:100030000C94D2010C94D2010C94D2010C94D201F4
:100040000C94D2010C94D2010C94D2010C94D201E4
:100050000C94D2010C94D2010C94D2010C940A0A93
:100060000C94D2010C94D2010C94D2010C94D201C4
:100070000C94D2010C94D2010C94D2010C94D201B4
:100080000C94540A0C94D2010C94D2010C94D20119
:100090000C94D2010C94D2010C94D2010C94D20194
:1000A0000C94D2010C94D2010C94D201D5F08D1491
:1000B000A1C881CFD9F1AF2000F0F89C8E8783874B
:1000C0008E9CF8F00000FEFF0303030303070EFC01
:1000D000F80000FEFF0303030303070EFCF8000013
:1000E000FFFF00000000000000FFFF0000FEFF8394
:1000F00083838383C7EE7C380000F8FC0E0703037C
:1001000003070EFCF800003F7FE0C08080C0E07F66
:100110003FFFFF01010101010101FFFF0000FFFF9F
:100120000C0C0C0C1C3E77E3C100007FFFC0C0C06C
:10013000C0C0E0703F1F00001F3F70E0C0C0C0E0C3
:10014000703F1F00007FFFC1C1C1C1C1E3773E1CEA
:1001500000001F3F70E0C0C0C0E0703F1F00000003
:10016000000001FFFF010000000A4869676873632F
:100170006F72650A000A001E003C0064009600C809
:10018000005072657373204120746F20706C617928
:1001900020616761696E2100596F75207365742055
:1001A00061206E6577206869676873636F72652187
:1001B0000000081C361C08000000143E143E140009
:1001C0000000183C7E3C180000003C3C3C3C3C00DD
:1001D00000003C56EB563C00003E362A362A362AB2
:1001E0003E80C0E0F0F8FCFEFFFFFEFCF8F0E0C04F
:1001F000800103070F1F3F7FFFFF7F3F1F0F070394
:1002000001507265737320537461727400496E7388
:1002100065727420436F696E00080B0002020200D1
:10022000000904000001020200000524001001057D
:1002300024010101042402060524060001070581AA
:100240000310004009040100020A00000007050233
:100250000240000007058302400000040309041265
:10026000010002EF020140412336000001010203B8
:100270000141726475696E6F204C4C430041726499
:1002800075626F79001F051F1F151B1F11111F11AC
:100290000E1F15111F05011F111D1F041F001F0038
:1002A00010101F1F041B1F10101F061F1F011F1FF0
:1002B000111F1F05071F311F1F051B17151D011FCC
:1002C000011F101F0F100F1F0C1F1B041B071C0703
:1002D0001915130C121E1F120C1E12120C121F0CD9
:1002E0001A14041F052E2A1E1F021C001D00201DAB
:1002F000001F041A011F001E041E1E021E1E121ED5
:100300003E120C0C123E1E020614120A020F121E9E
:10031000101E0E100E1E081E1A041A2E281E1A1267
:10032000161F111F001F001D151711151F07041F91
:1003300017151D1F151D01011F1F151F17151F0064
:10034000170000100004040401000A006400E80320
:100350001027350B11241FBECFEFDAE0DEBFCDBF73
:1003600011E0A0E0B1E0EEE2F7E202C005900D92EC
:10037000A833B107D9F726E0A8E3B1E001C01D9288
:10038000A035B207E1F711E0CAEAD1E004C0219735
:10039000FE010E948F13C93AD107C9F70E94580B7A
:1003A0000C9495130C94000090E121E061FD24E091
:1003B00060FD220F62FD2295687F969FD001112477
:1003C000A80FA151BE4F8C91822B8C930895AF92B0
:1003D000BF92CF92DF92EF92FF920F931F93CF9332
:1003E000DF936B01EC015C01A40EB11C7B01E20EFA
:1003F000F11CCA15DB05DCF48601D7FE02C010E053
:1004000000E0C70121E4E216F10414F080E490E07A
:100410000817190754F4C038D10520F4B801CE01EB
:100420000E94D4010F5F1F4FECCF2196E2CFDF91E6
:10043000CF911F910F91FF90EF90DF90CF90BF90E1
:10044000AF90089580E0EFEEF1E081118FEF00248E
:1004500081938193819381930394D1F70895EFEE73
:10046000F1E0A0E0B8E000800EBC8111012C1197F2
:10047000A0FDFDCF0192B9F70DB40895FC01809164
:10048000EE01882311F13FB7F89482E08093E900F0
:100490002091F200822F90E01816190614F481E0E2
:1004A00090E0882339F0289844E64093ED0140918C
:1004B000F1004083222339F02091F200211103C082
:1004C0002BE62093E8003FBF08958FEF9FEF08953C
:1004D0002FB7F89483E08093E9009091E800892F8A
:1004E000807295FF04C09091F20080E4891B2FBFB9
:1004F00008958091E50181110DC082E08093E101B2
:1005000084E08093E2011092E4011092E30181E023
:100510008093E50181EE91E00895CF93DF931F92E0
:10052000CDB7DEB76983DC01ED91FC910280F381E8
:10053000E02D41E050E0BE016F5F7F4F09950F90C5
:10054000DF91CF91089583E08093E9008091F200DC
:10055000882319F08AE38093E80008950E946802D6
:1005600090E00895CF93DF931F92CDB7DEB7FC01E3
:100570008485958597FD08C02FEF3FEF3587248749
:100580000F90DF91CF910895CE0101960E943E0217
:10059000019719F4898190E0F3CF8FEF9FEFF0CFAF
:1005A0000F931F93CF93DF931F92CDB7DEB78C01CC
:1005B000FC018485958597FF0BC0CE0101960E94B2
:1005C0003E02019771F4898190E0F8019587848754
:1005D000F801848595850F90DF91CF911F910F9140
:1005E00008958FEF9FEFF1CFFC018485958597FDEE
:1005F0000BC09FB7F89482E08093E9008091F200ED
:100600009FBF90E0019608959FB7F89482E0809391
:10061000E9008091F2009FBF90E008954091DB01D6
:100620005091DC012091D9013091DA014217530732
:10063000B4F49091E8009570E1F39091E80092FD98
:1006400019C08093F1008091DB019091DC0101964B
:100650008F739927892B19F48EEF8093E80080918E
:10066000DB019091DC0101969093DC018093DB012A
:1006700081E0089580E00895DF92EF92FF920F935A
:100680001F93CF93DF93D82E8A01EB017B01E40EF9
:10069000F51ECE15DF0559F0D7FE12C0FE0184917C
:1006A0000E940E0321968111F4CF0FEF1FEFC801B6
:1006B000DF91CF911F910F91FF90EF90DF90089500
:1006C0008881EECF0F931F93CF93DF931F92CDB707
:1006D000DEB782E0898342E450E069E172E080E8BD
:1006E0000E943C030E947902DC0112960D911C913C
:1006F0000115110589F0D801ED91FC910280F3817B
:10070000E02DBE016F5F7F4FC801099597FD04C0C2
:10071000F80100851185ECCF89810F90DF91CF9191
:100720001F910F910895615030F02091F100FC016C
:1007300020830196F8CF289884E68093ED010895F0
:100740000E94AB03982F0C94AB030DB407FEFDCFB2
:100750008EB5599A08950DB407FEFDCF8EB51EBC17
:10076000089590E0409F09F4142E5527090E151E98
:10077000600D711D851F11240C94CA0359980E94A5
:10078000D603862F0E94D603852F0E94D603842F7E
:100790000C94D603462F50919101570F609192010E
:1007A000681F83E00E94BE031EBC08958EBD00003A
:1007B0008EB50DB407FEFCCF08953FB7F894809135
:1007C0008D0190918E01A0918F01B091900126B57D
:1007D000A89B05C02F3F19F00196A11DB11D3FBF79
:1007E000BA2FA92F982F8827BC01CD01620F711D48
:1007F000811D911D42E0660F771F881F991F4A9542
:10080000D1F708958F929F92AF92BF92CF92DF92CD
:10081000EF92FF926B017C010E94DD034B015C01B2
:10082000C114D104E104F104B9F00E94DD03681998
:1008300079098A099B09683E73408105910580F317
:1008400081E0C81AD108E108F10828EE820E23E001
:10085000921EA11CB11CE4CFFF90EF90DF90CF90CF
:10086000BF90AF909F908F9008958F929F92AF927C
:10087000BF92CF92DF92EF92FF920F931F93CF938D
:10088000DF936C017B018A0180910E01882309F4BA
:100890005CC08091EE01882309F457C08091E0018B
:1008A00080FF05C08091E00082608093E000E80155
:1008B000B12C8AEFA82E93E0892E2AE3922E20975E
:1008C00011F4BB20D9F10E94680281110AC0AA94D8
:1008D000AA20D9F161E070E080E090E00E9402047B
:1008E000EECF8C171D0611F00CF08C2F9FB7F894EB
:1008F0008092E9002091E80025FD02C09FBFDFCF74
:10090000282F30E0C21BD30BF701815020F041911A
:100910004093F100FACFE20EF31EBB2021F090923B
:10092000E800B12CEBCF8091E80085FDE7CF9092F5
:10093000E800BB24B394209709F3F3CF5D9884E6D5
:100940008093DF01101611063CF081E090E0F60183
:100950009383828310E000E0C801DF91CF911F9163
:100960000F91FF90EF90DF90CF90BF90AF909F904E
:100970008F9008952D9A0895BC0190E080E00C942A
:1009800002048FB18095807F669B88601C9B846089
:10099000089590919A01982329F490919B019823AE
:1009A00081E009F480E00895CF93C82F0E94C1042C
:1009B000982F9C2381E09C1380E0CF9108953F9273
:1009C0004F925F926F927F928F929F92AF92BF925F
:1009D000CF92DF92EF92FF920F931F93CF93DF930B
:1009E00030E0F901E80FF91F1E161F060CF0D7C002
:1009F000803891050CF0D3C0FB01E00FF11D1E16ED
:100A00001F060CF0CCC0603471050CF0C8C0DB01CF
:100A100077FF04C0AA27BB27A61BB70BA770BB276D
:100A2000FB0177FD3796C3E0F595E795CA95E1F7A9
:100A300077FF07C0319768E070E0EB01CA1BDB0B62
:100A4000DE01402E469446944694512C077019F0CE
:100A5000DFEF4D1A5D0ABF01EF01D695DC2FCC27E1
:100A6000D795C795C80FD91FC151DE4F8A01460ED1
:100A7000571E48E050E04A018A1A9B0A6415750522
:100A800009F48DC06830710509F489C06F3FEFEF3C
:100A90007E070CF44BC06C0150E040E03E01E0E802
:100AA0006E0E711CD7FC35C06F3F760709F473C01A
:100AB0005E01A40EB51EF501F080FA01E00FF11FF2
:100AC00033243394E31039C0E4910A2E01C0EE0FB1
:100AD0000A94EAF7FE2AF501F0821097D1F0673008
:100AE0007105B9F05301A40EB51EF501F080FA01AD
:100AF000E00FF11F33243394E31035C0E491F0E0AC
:100B0000082C02C0F595E7950A94E2F7FE2AF50154
:100B1000F0824F5F5F4FFFEFCF1ADF0A4217530794
:100B20002CF4F0E8CF16D10409F0BCCF6F5F7F4FF3
:100B3000C058DF4F020F131FA1CFE1100CC0E4918A
:100B4000F0E00A2E02C0EE0FFF1F0A94E2F7E095D4
:100B5000F095FE22C0CFE4910A2E01C0EE0F0A9458
:100B6000EAF7FE26B8CFE1100CC0E491F0E0082CC3
:100B700002C0F595E7950A94E2F7E095F095FE221C
:100B8000C6CFE491F0E0082C02C0F595E7950A94F1
:100B9000E2F7FE26BCCF109709F0A4CFBACFDF91C1
:100BA000CF911F910F91FF90EF90DF90CF90BF906A
:100BB000AF909F908F907F906F905F904F903F90FD
:100BC0000895CF92DF92EF92FF920F931F93CF93EE
:100BD000DF936C01C0E5D3E0F12C14E044E3FE01A7
:100BE00085919491C816D90638F0FE0185919491AB
:100BF000C81AD90A4F5FF3CF81E0443309F480E08B
:100C0000F82A11F411111EC083E04802A00111243A
:100C10004B575D4F60911101062E000C770B8091B0
:100C20000F01E090120106E023E0082E000C990B62
:100C30000E94DF04809113018D5F90910F01890F55
:100C400080930F01115022971F3F09F0C7CFDF910A
:100C5000CF911F910F91FF90EF90DF90CF9008956B
:100C6000EF920F938A33BCF48033BCF5813209F4E0
:100C700044C05CF48A3099F1809113018D5F9091AA
:100C80000F01890F80930F0135C08D32C1F18E3273
:100C900099F78FE309C081347CF38B35E4F09FE949
:100CA000980F87549A3140F793E08902A0011124EC
:100CB0004B575D4F60911101062E000C770B809110
:100CC0000F01E090120106E023E0082E000C990BC2
:100CD0000E94DF04D1CF8154E7CF8C5FE5CF8091B4
:100CE000100180930F018091110190911401890FDF
:100CF000809311010F91EF9008958EE3D5CF80E49A
:100D0000D3CF0F931F93CF938C01C0E0F801EC0F6A
:100D1000F11D8491882329F084910E943006CF5FD1
:100D2000F5CFCF911F910F910895CF93C09193016B
:100D3000CC2331F080913C0110923C018F3F19F49B
:100D40008C2FCF91089580919301882309F42FC0AF
:100D50008091880181112BC06091390170913A0115
:100D600080913B010E94CA03EBE5F1E02EE230E006
:100D70002150304021F00E94AB038193F9CF0E94B3
:100D8000A50380833FE0EBE5F1E090E080E0219176
:100D900041915191452B11F4109293012695821B9C
:100DA00091093150A1F790938A0180938901809134
:100DB0009301811106C0109271001092C10010922F
:100DC000930180918801882309F4BACF81508093E0
:100DD00088018111B5CF8091390190913A01A0919C
:100DE0003B018E96A11D8093390190933A01A09307
:100DF0003B01A6CFFF920F931F93CF93DF93C1E7E1
:100E0000D0E0188201EC10E0F801108210929301FA
:100E10006093390170933A0180933B0110928801ED
:100E2000FF24F394F09293010E94950680E094E0F1
:100E300090939900809398001092950010929400DE
:100E4000F801F08282E08883DF91CF911F910F91AA
:100E5000FF900895EF92FF920F931F93CF93DF932C
:100E6000E82EF12C10E000E0D0E0C0E00E151F05E8
:100E7000B9F0C801805A9C4F0E94FB12C82788E035
:100E80009E0121703327D695C795232B21F091E041
:100E9000C92790EAD927815099F70F5F1F4FE6CFF6
:100EA000CE01DF91CF911F910F91FF90EF900895A8
:100EB00082E090E00E94FB12882331F03E9A3F9A34
:100EC00081E080938B01089510928B013E983F98AA
:100ED00008951F920F920FB60F9211248F939F9334
:100EE0008091E1009091E100937F9093E10083FF76
:100EF0000FC01092E90091E09093EB001092EC008B
:100F000092E39093ED001092EE0198E09093F00040
:100F100082FF22C093E09093E9009091F200992320
:100F200019F09AE39093E8009091DF01992341F042
:100F30009091DF0191509093DF01911101C05D9A72
:100F40009091ED01992341F09091ED019150909392
:100F5000ED01911101C0289A84FF18C08091E20030
:100F60008E7E81608093E2008091E1008F7E80938D
:100F7000E1008091E0018E7E80618093E0019F918D
:100F80008F910F900FBE0F901F90189580FFF7CF95
:100F90008091E2008E7E80618093E2008091E1008A
:100FA0008E7E8093E1008091E0018E7E8160E5CFAE
:100FB0001F920F920FB60F921124CF92DF92EF92F1
:100FC000FF920F931F932F933F934F935F936F93D2
:100FD0007F938F939F93AF93BF93EF93FF93CF93A1
:100FE000DF93CDB7DEB76C97DEBFCDBF1092E900BF
:100FF0008091E80083FF25C068E0CE0145960E94FD
:10100000930382EF8093E8008D8987FF39C0909128
:10101000E80090FFFCCF982F907609F034C19E89AC
:101020004F89588D2F89F88C911131C0803861F526
:101030008091DE018093F1001092F1008EEF809399
:10104000E8006C960FB6F894DEBF0FBECDBFDF91FF
:10105000CF91FF91EF91BF91AF919F918F917F9130
:101060006F915F914F913F912F911F910F91FF9041
:10107000EF90DF90CF900F900FBE0F901F901895BC
:101080009EEF9093E800C7CF1092F100D5CF91303A
:1010900059F48111D3CF4130510581F68091DE01A1
:1010A0008D7F8093DE01CACF933049F48111C6CF82
:1010B0004130510519F68091DE018260F2CF953002
:1010C00041F48091E80080FFFCCF20682093E3008A
:1010D000B5CF963009F0A9C00B8D1C8D22E010927F
:1010E000E9001092DC011092DB01F2122EC0109286
:1010F000DA011092D9010E9462031F8299E099835C
:10110000FA8291E09E8390EA98879AEF99872091DE
:10111000DB013091DC01275F3F4F3C832B838D83C4
:101120001092E9001092DC011092DB011093DA01B9
:101130000093D90149E050E0BE016F5F7F4F80E02E
:101140000E943C030E94620379CF1093DA0100935E
:10115000D9010E947902DC0112960D911C910115B2
:10116000110509F451C1D801ED91FC910480F5817C
:10117000E02DBE016B5E7F4FC8010995009709F015
:101180003EC1F80100851185EACFF3E0FF120EC0E1
:101190008F89882309F440C0823061F440E867E019
:1011A0008DE792E00E94020B811148CF81E280938B
:1011B000EB0047CF813029F440E86BE081E792E013
:1011C000F1CF833099F70E947902DC011296ED90FD
:1011D000FC908E010F5F1F4F6801E114F10479F05C
:1011E000D701ED91FC910680F781E02DB801C70190
:1011F0000995080F111DF701E084F184EECFD801A5
:101200001C92F60101900020E9F73197BF016C199B
:101210007D0940E0C601C6CF6BE572E0FB01449159
:1012200050E080E80E943C0309CF973009F4BECF1C
:10123000983021F481E08093F10000CF993009F0DB
:10124000FDCE837009F0B2CFEAE1F1E081E031E058
:1012500096E32191222371F08093E9003093EB0013
:10126000DF0111972C912093EC009093ED008F5F9C
:10127000873079F78EE78093EA001092EA008F8931
:101280008093EE01DBCE8B8D9C8D1092E900109245
:10129000DC011092DB019093DA018093D901898DF2
:1012A000811192C08E899D89913A49F4813209F069
:1012B0007DCF47E050E067E071E080E0B3CF91324E
:1012C00009F074CF833269F48F89988DB0E0A0E083
:1012D0008093030190930401A0930501B09306014C
:1012E000ADCE803269F48091E80082FFFCCF67E0E8
:1012F00087E091E00E9493038BEF8093E8009ECEFD
:10130000823209F09BCE8F8980930E01EEEFFFE7CA
:10131000859194918B3F9C4D51F1E0E0F8E08091F4
:10132000070190910801A0910901B0910A01803B49
:101330009440A105B105F1F480910E0180FD1AC021
:10134000EE3F8AE0F80789F587E797E79183808386
:10135000809160008093DD0188E19BE00FB6F894F6
:10136000A895809360000FBE9093600067CEEEEF6B
:10137000FAE0D5CF808191818737974709F05ECE1B
:10138000A895809160008861809360008091DD0164
:1013900080936000EE3F2AE0F20789F08091FE0A18
:1013A0009091FF0A9183808349CE80819181873714
:1013B000980751F29093FF0A8093FE0AC5CF1092CE
:1013C000FF0A1092FE0A3ACE0E947902DC011296C0
:1013D0000D911C910115110509F4E8CED801ED918C
:1013E000FC910190F081E02DBE016B5E7F4FC80142
:1013F0000995811123CEF80100851185EBCF1816D0
:1014000019060CF41BCED2CEF1E0FF12BECE6FE572
:1014100072E004CF1F920F920FB60F9211242F93F8
:101420003F938F939F93AF93BF9380919601909139
:101430009701A0919801B091990130918C0123E01E
:10144000230F2D3758F50196A11DB11D20938C0156
:101450008093960190939701A0939801B09399017E
:1014600080918D0190918E01A0918F01B09190019A
:101470000196A11DB11D80938D0190938E01A093C3
:101480008F01B0939001BF91AF919F918F913F9148
:101490002F910F900FBE0F901F90189526E8230FE5
:1014A0000296A11DB11DD2CF1F920F920FB60F92BF
:1014B0001124EF92FF920F931F932F933F934F931B
:1014C0005F936F937F938F939F93AF93BF93CF93CC
:1014D000DF93EF93FF9380918B01882309F452C02F
:1014E00080919301882309F44DC0C0919800D09158
:1014F0009900D695C795D695C79560918901709149
:101500008A019FE0F92EEBE5F1E0ADE3B1E08FEF6A
:101510009EE3E190419151918A01E11050C01296F1
:10152000FA94F110F6CF4091D301469F9001479F66
:10153000300D1124359527953595279535952795A7
:1015400035952795880F991F880F991F813044E0A2
:10155000940708F450C0019788279C7F9C5F909364
:10156000990080939800293731050CF047C028383E
:101570008FEF38070CF444C020581092BF0020931E
:10158000CF0006C08FEF9FEF909399008093980053
:10159000FF91EF91DF91CF91BF91AF919F918F918B
:1015A0007F916F915F914F913F912F911F910F917B
:1015B000FF90EF900F900FBE0F901F9018952D91F8
:1015C0003C9111972C0F3D1F2417350710F0241B59
:1015D000350B569547952417350718F46E0D711D78
:1015E0008A012D933D93021B130B0817190708F06E
:1015F00097CFC80195CF80E094E0B1CF28E7BCCF6A
:1016000028E8BACFEF92FF920F931F93CF93DF9307
:10161000F82E192FE62E042F81E0860F880F0E94E6
:101620000E0383E00E940E03CF2DD12FEC0EFD2E72
:10163000F11CCE15DF05B9F007FF13C0FE01849140
:101640000E940E03182F80E00E940E038123219632
:101650008111EFCFDF91CF911F910F91FF90EF900C
:1016600008958881EDCF81E0F5CFEFEEF5E01382AC
:10167000128288EE93E0A0E0B0E084839583A68395
:10168000B78384E291E0918380838FEF9FEF95870A
:10169000848782E693E090934F0680934E06EFE3B3
:1016A000F6E088E390E0938382831586168608959A
:1016B000CF93DF9300D000D01F92CDB7DEB77894E0
:1016C00084B5826084BD84B5816084BD85B5826047
:1016D00085BD85B5816085BD80916E0081608093F8
:1016E0006E00109281008091810082608093810061
:1016F0008091810081608093810080918000816071
:10170000809380008091910082608093910080910D
:10171000910081608093910080919000816080931E
:1017200090008091C10084608093C1008091C100CD
:1017300082608093C1008091C10081608093C1006C
:101740008091C30081608093C3008091C00082605B
:101750008093C0008091C20081608093C20080911C
:101760007A00846080937A0080917A00826080930E
:101770007A0080917A00816080937A0080917A006B
:10178000806880937A001092EE011092DE01109230
:10179000E0018091D70081608093D70080EA809338
:1017A000D80089B5806189BD89B5826089BD09B4D9
:1017B00000FEFDCF61E070E080E090E00E94020456
:1017C0008091D8008F7C80618093D8008091E00068
:1017D000807F8093E0008091E1008E7E8093E10025
:1017E0008DE08093E200559A209A81EC80937C00F2
:1017F00085B1806F85B984B1877E84B984B1876EE5
:1018000084B95E9A5F988AB1806D8AB9769A6E982B
:1018100081B3806F81BB899880B38D7080BB80E578
:101820008CBD81E08DBD85E090E00E94BC045F9A94
:1018300085E090E00E94BC045E985C98ECEAF0E0E1
:1018400084918EBD00000DB407FEFDCF319620E0DF
:10185000E93BF207A9F75C9A81E8809364008091E4
:10186000650081608093650080E00E942F0280E81F
:101870000E94D4048823A9F05C9885EA8EBD0000FC
:101880000DB407FEFDCF5C9A2E982F982D9880916D
:10189000640080628093640081E083BF889513BEFA
:1018A000FCCF84E00E94D404882309F448C02D981A
:1018B00084E80E94D4048823E1F00E94BA0488ECF2
:1018C00090E00E94BC042F9882E090E00E94FB12FE
:1018D0008F3F29F06FEF82E090E00E94091384EFC0
:1018E00091E00E94BC042F9A84E80E94D4048111E4
:1018F000FBCF84E10E94D4048823E1F00E94BA0463
:1019000088EC90E00E94BC042E9882E090E00E9457
:10191000FB12882329F060E082E090E00E94091326
:1019200084EF91E00E94BC042E9A84E10E94D404CA
:101930008111FBCF88EC90E00E94BC04B2CF0E94E2
:10194000BA040E94580781E090E00E94FB12182F11
:10195000147081E090E00E94FB1281FF10C0111111
:101960002E9881EF9FEF9C838B8380E40E94D404A8
:10197000882309F484C02E9A2F9A0E94BA0482E325
:1019800090E00E94BC040E94C1048111F8CF80E164
:10199000809300010E9422025E9AE4E1F0E086EB6F
:1019A00098EF25913591559145912851354909F484
:1019B000CA01809391019093920159988BEA0E94F9
:1019C000D603599A0E945807109271001092C100D4
:1019D0001092930186E582BF82E48093C00081E08B
:1019E0008093C30080E48093C4001092BF008FE70F
:1019F0008093D1001092900089E08093910085E05F
:101A00008093D30180914E0690914F060E9403135C
:101A10009C838B8382E00E942A07EB81FC81E8177C
:101A2000F90741F480E693E00E9403139093470680
:101A300080934606ACE32A2E312CB4E08B2E912CF9
:101A4000A12CB12C13E0412E512C612C712C8FB79D
:101A5000F89440919601509197016091980170918E
:101A600099018FBF809194018823E1F11092940134
:101A700080E090E0892B59F30E940000E8CF112309
:101A800031F0EB81FC81349711F42E9A2F9881E08C
:101A90000E942F02EE24E39400E128E549EB50E098
:101AA0006B817C8184E190E00E94DF0480E00E94F1
:101AB0002F028FE090E00E94BC042B813C812F5FBD
:101AC0003F4F3C832B832931310509F04ECF112341
:101AD00011F02F9A2D9880E991E00E94BC040E9499
:101AE000BA044DCF80919501F42FF81B8F2F909160
:101AF0000001F91748F48F5F891708F0B9CF81E02A
:101B000083BF889513BEB4CF81E080939401409346
:101B100095018091D5019091D60101969093D601BF
:101B20008093D5018091020181110E94220259986F
:101B300085E00E94D60380E00E94D60380FDFBCFA3
:101B4000599A0E94950681111BC08091D801882363
:101B5000B9F00E94A312A50194010E942C13462FF4
:101B600003E020E066E579E487E00E94B1030E948B
:101B7000A003782F0E94A503682F892F0E94FA06E0
:101B800020919B012D8320939A010E94C104809390
:101B90009B0180910201813071F160F0823009F483
:101BA00010C1833009F4F4C35E9880E00E942F02D4
:101BB0005E9A5ECF3091D7013B8337FD15C0832FEE
:101BC00090E0AC01F6E0440F551FFA95E1F7EE24E2
:101BD000E39400E421E070E060E00E94DF049B8178
:101BE0009F5F9093D701E0CF8B81853AC0F381E06E
:101BF00080930201F4CF8093120183E3809310015C
:101C000080930F0184E1809311011B822B81E22FCD
:101C1000F0E0EE5CFE4F8081181634F40E9430062E
:101C20003B813F5F3B83F2CF8091D50185FF5EC052
:101C3000109212018091D401813009F468C008F437
:101C400059C0823009F46EC088E00E94C90488231C
:101C500029F08091D4018F5F8093D40180E40E94A9
:101C6000C904882349F08091D301883028F48091F9
:101C7000D3018F5F8093D30180E20E94C90488233F
:101C800049F08091D301882329F08091D3018150BC
:101C90008093D301FF24F3948091D3018F1508F42E
:101CA00083CF8F2D90E08C010A5C1F4F000F111F16
:101CB000F101E81BF90BFC83EB83F7FF02C01C82E8
:101CC0001B822B813C812C33310509F478C000380C
:101CD000110534F437FD04C0B901C8010E94D401D4
:101CE0008B819C8101969C838B83EBCF81E08093D9
:101CF0001201A0CF87E28093100180930F0180E250
:101D0000809311018DE092E00E9481069DCF87E2D1
:101D10008093100180930F0180E28093110181E094
:101D200092E0F2CF8093020181E0809312018091D2
:101D3000D801811140C0809164008E7F809364003F
:101D400080917A00806480937A0080917A0086FD89
:101D5000FCCF00917800109179000E94DD0330E003
:101D600020E0980111270027600F711F821F931F29
:101D70002091640021602093640061157105810544
:101D8000910511F00E94F2120E94A312A501940184
:101D90000E942C13462F03E020E066E579E487E0FB
:101DA0000E94B1030E94A003782F0E94A503682F10
:101DB000892F0E94FA0681E08093D80145CFF394E1
:101DC0006BCF80E40E94D4048B8380E20E94D40411
:101DD000EB81E81BFF0BCF0120913F0630914006BD
:101DE000820F931F97FD14C29093400680933F0685
:101DF00080913F06909140068937910534F088E73D
:101E000090E09093400680933F06F0914306FF5F79
:101E1000F0934306F595FB8388E00E94D40420915B
:101E2000410630914206882361F08D8183FDF5C122
:101E30002833310509F0F1C188EF809343069CEF08
:101E40009B838B81280F311D87FD3A9529333105FE
:101E50000CF0E9C130934206209341062091010124
:101E600030E080E890E0821B930B97FD01969595FA
:101E70008795409141065091420660913F067091CE
:101E80004006FB0138968E179F0794F5820F931F2B
:101E9000681779076CF5445351094C30510540F5EA
:101EA0008091480690914906A0914A06B0914B0650
:101EB00022E330E0309342062093410622EF209344
:101EC0004306892B8A2B8B2B99F42FB7F89480919A
:101ED000960190919701A0919801B09199012FBF1F
:101EE0008093480690934906A0934A06B0934B0608
:101EF0008091480690914906A0914A06B0914B0600
:101F0000892B8A2B8B2B09F49CC0EAEBF1E0FC8334
:101F1000EB8313EDE12E11E0F12E12E001E084E1FC
:101F2000C82EEB81FC818481823009F092C18091BE
:101F3000430618160CF07BC041815081852F052E79
:101F4000000C990B209141063091420660913F06AA
:101F500070914006FB0138968E179F070CF067C002
:101F60000896681779070CF062C0842F042E000CC5
:101F7000990BB901685F7F4F861797070CF057C020
:101F8000BC01685F7F4F261737070CF050C0F8EF91
:101F9000F09343060A979093420680934106EB81A3
:101FA000FC81A3818A2FA23091F480914D06882371
:101FB00041F080914C068F5F833008F03DC18093E3
:101FC0004C06E0914C0682E08E0FC0924D06EB81EC
:101FD000FC810483E82FF0E0EE0FFF1FEB58FE4F6B
:101FE000659174918091440690914506860F971FE4
:101FF0009093450680934406ECE9F1E030E020E060
:10200000858181111EC186E0829FF001839FF00DC2
:102010001124E456FE4F92E39583538344837183E6
:102020006083A23009F00BC180914C0682832B8122
:102030003C812B5F3F4F3C832B83E216F30609F074
:1020400070CF80914D06882339F0815080934D06E2
:10205000811102C010924C066091410670914206B7
:1020600028E048E080913F06909140060E94E701F9
:102070001092100110920F011092110180914406EC
:10208000909145060E94E10589E691E00E94810653
:1020900080914606909147060E94E105809148068E
:1020A00090914906A0914A06B0914B06892B8A2B44
:1020B0008B2B79F187E78093100180930F011092A9
:1020C00011012FB7F8948091960190919701A091FA
:1020D0009801B09199012FBF40914806509149064F
:1020E00060914A0670914B06841B950BA60BB70BAB
:1020F000EAE0B695A79597958795EA95D1F7F1010E
:10210000E81BF90BCF011E161F060CF0EFC00E9452
:10211000E1058091480690914906A0914A06B09148
:102120004B06892B8A2B8B2BA9F12AEB31E03C83C0
:102130002B8373EDC72E71E0D72EEB81FC81948148
:10214000992301F180812281820F8083913009F0EF
:10215000D5C06181062E000C770B65507109082EE1
:10216000000C990BEE24E39400E120E141EE51E0F4
:1021700005970E94DF04EB81FC818381823009F0A6
:10218000B9C084838B819C8105969C838B83C81600
:10219000D90699F68091D501811107C0809101017E
:1021A000863018F08150809301014091010180E850
:1021B00090E0841B910997FD019625E06BE370E0A8
:1021C000959587950E94E701ECE9F1E0FC83EB83AC
:1021D0000AEB11E0EB81FC81F580FF2009F4CDC012
:1021E000948183818093100180930F01909311015A
:1021F000808191810E94E105E12CEB81FC8182814B
:10220000E81608F0B6C081E20E943006E394F5CFEC
:102210001092400610923F06EBCDEB81E7FD11CE08
:10222000F1E0FB830ECE88E390E09093420680932A
:1022300041061092430612CEA0934C06C2CE1282E3
:10224000F6CE2F5F3F4F36962530310509F0D8CEB8
:10225000EECE8111ECCE0E94A31220E230E040E0ED
:1022600050E00E942C13672B682B692B09F0DFCEFE
:10227000EB81FC8114830E94A31222E030E040E055
:1022800050E00E942C13D62E679566276795EB8148
:10229000FC8160830E94A3122BE230E040E050E01A
:1022A0000E942C13685F7F4F8F4F9F4FEB81FC8103
:1022B000618381E0D1108FEFEB81FC8182830E94EA
:1022C000A31228E030E040E050E00E942C13EB81A4
:1022D000FC816383611102C01383A9CEEB81FC8171
:1022E000663010F00383A3CE1382A1CE83E08093E7
:1022F00002010FCFEB81FC81148244CFEB81FC8182
:102300009381923081F487FD03C0818189375CF02D
:102310000E94A312A30192010E942C13EB81FC8165
:102320008381861B83838091D50183FB882780F975
:1023300089831A82EB81FC81438150E0440F551F51
:1023400029813A81420F531F440F440F440F50E03C
:102350004F545E4F6181062E000C770B8081EE2476
:10236000E39408E028E0082E000C990B0E94DF049B
:1023700009CFFA94EB81FC81F5822B813C812A5FA5
:102380003F4F3C832B830217130709F023CF0CCC5C
:102390001092100110920F011092110180914406C9
:1023A000909145060E94E1058091100180930F01F4
:1023B0008091110190911401890F80931101209156
:1023C0004406309145068091460690914706821753
:1023D000930778F488E991E00E94810680911001CA
:1023E00080930F018091110190911401890F8093C6
:1023F000110181E891E00E94810688E00E94C904F1
:10240000882309F4D1CB60914406709145068091F0
:102410004606909147068617970790F470934706F3
:102420006093460680E693E00E94171382E00E94C4
:102430002A07BC0180914E0690914F060E94171307
:102440000E94220281E0809302011092D401109236
:10245000400610923F0688E390E0909342068093F6
:1024600041061092430610924506109244061092BF
:1024700048061092490610924A0610924B0683E2D3
:10248000809301011092A1011092A7011092AD0159
:102490001092B3011092B9011092BE011092C301C3
:1024A0001092C8011092CD011092D2017DCB8F9273
:1024B0009F92AF92BF92CF92DF92EF92FF92CF9313
:1024C000DF93EC01688179818A819B8161157105B7
:1024D0008105910521F464E279ED8BE597E02DE12A
:1024E00033EF41E050E00E942C1349015A019B0157
:1024F000AC01A7EAB1E40E944B136B017C01ACEE86
:10250000B4EFA50194010E945913C60ED71EE81E10
:10251000F91EF7FE06C081E0C81AD108E10880E87C
:10252000F80AC882D982EA82FB82C701B6019F7786
:10253000DF91CF91FF90EF90DF90CF90BF90AF9061
:102540009F908F9008958F929F92AF92BF92CF925B
:10255000DF92EF92FF9260911501709116018091C8
:10256000170190911801611571058105910521F4FC
:1025700064E279ED8BE597E02DE133EF41E050E047
:102580000E942C1349015A019B01AC01A7EAB1E456
:102590000E944B136B017C01ACEEB4EFA5019401DA
:1025A0000E945913C60ED71EE81EF91EF7FE06C07C
:1025B00081E0C81AD108E10880E8F80AC092150144
:1025C000D0921601E0921701F0921801C701B601EE
:1025D0009F77FF90EF90DF90CF90BF90AF909F904C
:1025E0008F900895609315017093160180931701E1
:1025F000909318010895F999FECF92BD81BDF89A84
:10260000992780B50895A8E1B0E042E050E00C942D
:102610001E13262FF999FECF1FBA92BD81BD20BD92
:102620000FB6F894FA9AF99A0FBE019608950E948F
:102630000913272F0C940A13DC01CB01FC01F99933
:10264000FECF06C0F2BDE1BDF89A319600B40D92FE
:1026500041505040B8F70895052E97FB1EF40094A2
:102660000E94431357FD07D00E945E1307FC03D05E
:102670004EF40C94431350954095309521953F4F5F
:102680004F4F5F4F089590958095709561957F4F5E
:102690008F4F9F4F08950E948013A59F900DB49F68
:1026A000900DA49F800D911D11240895B7FF0C94E7
:1026B0004B130E944B13821B930B0895A1E21A2E19
:1026C000AA1BBB1BFD010DC0AA1FBB1FEE1FFF1FD6
:1026D000A217B307E407F50720F0A21BB30BE40B26
:1026E000F50B661F771F881F991F1A9469F760956D
:1026F0007095809590959B01AC01BD01CF01089527
:10270000A29FB001B39FC001A39F700D811D112432
:10271000911DB29F700D811D1124911D0895EE0F22
:0E272000FF1F0590F491E02D0994F894FFCF6F
:10272E00102301FFFFFFFF00E1000000000000008A
:10273E0000000101080100000000C18081000000BE
:10274E00000000008D023504AE02A302F402B202B4
:08275E00D002426F696E6B00AE
:00000001FF
